:0A00000026C0FECFFDCFFCCFFBCFE2
:10000A00FACFF9CFF8CFF7CFF6CFF5CF4AC0F3CF73
:10001A00F2CFF1CFF0CFEFCFEECFEDCF1027E8033D
:10002A0064000A0001000010000110000100000035
:10003A000000000000000100020038000600040071
:10004A003A000000F894EE27ECBBF1E0FBBFEBBFEF
:10005A00E5BFF8E1F1BDE1BD8DE0A2E0BB27ED937C
:10006A008A95E9F780E094E0A0E6ED930197E9F735
:10007A00E0E4F0E085919591009761F0A591B59142
:10008A0005901590BF01F00105900D920197E1F7D7
:10009A00FB01F0CFEFE5EDBFE4E0EEBFC0E6D1E053
:1000AA0046C0EA93FA93EFB7EA93D4D01BB10CB1E6
:1000BA00E12FEC7179F4EB2DBDD00083B394E8E025
:1000CA00EB1509F4BB24D394E8E0ED1519F4DD240B
:1000DA00689420F8C2D0E991EFBFF991E991189597
:1000EA001A93DD20F1F3EA2DA5D01081A394E8E05C
:1000FA00EA1509F4AA24F894DA947894E12F19916C
:10010A000895552011F0A89A03C0552009F4A8981B
:10011A00442011F0A99A03C0442009F4A998772031
:10012A0011F0AA9A03C0772009F4AA980895E0E08A
:10013A00E8BBE7BBE5BBE7E0E4BBE0E0E2BBE1BB71
:10014A00E3BFE2BFEFBDEEBDEDBDECBDE7BDE6BD71
:10015A00EBBDEABDE9BDE8BDE2BDE5BDE4BDE3BD79
:10016A00E5BFE9BFEBB9E0E9EAB9E6E8E0BDE0E0FE
:10017A00E0BDE7E6E9B9E0E8E8B9E0E0E0BF789495
:10018A00A898A998AA98552011F0A89A03C05520B2
:10019A0009F4A898442011F0A99A03C0442009F44C
:1001AA00A998772011F0AA9A03C0772009F4AA988F
:1001BA00082C092849F0F40131974F01E1E0F0E0F9
:1001CA00FA93EA933BD034C0082C092889F5E8EC65
:1001DA00F0E04F016624DD2059F182DF6E2EE1E462
:1001EA00E61549F4552011F0552404C0552011F4A0
:1001FA00E1E05E2E17C0E2E4E61549F4442011F06E
:10020A00442404C0442011F4E1E04E2E0BC0E3E480
:10021A00E61541F4772011F0772404C0772011F411
:10022A00E1E07E2E6EDFDD2019F05ADF6E2EFBCF65
:10023A00AACFFFCFF0E0E05AFE4F0895E991F99175
:10024A00309639F088EE93E00197F1F7A895319747
:10025A00C9F708951A930A9308950991199108956F
:00000001FF
